:100000000C9446000C9465000C9465000C946500FB
:100010000C9465000C9465000C9465000C946500CC
:100020000C9465000C9465000C9465000C946500BC
:100030000C9465000C9465000C9465000C946500AC
:100040000C9465000C9465000C9465000C9465009C
:100050000C9465000C9465000C9465000C9465008C
:100060000C9465000C9465000C9465000C9465007C
:100070000C9465000C9465000C9465000C9465006C
:100080000C9465000C9465000C94650011241FBE4F
:10009000CFEFD0E1DEBFCDBF11E0A0E0B1E0EEE0F8
:1000A000F1E000E00BBF02C007900D92A030B10755
:1000B000D9F711E0A0E0B1E001C01D92A030B10776
:1000C000E1F70E9471000C9485000C94000020EF71
:1000D00030E004C0F9013197F1F701970097D1F7AB
:1000E0000895A59A20EF30E0AD9A88EE93E0F901EB
:1000F0003197F1F70197D9F7AD9888EE93E0F901C0
:0E0100003197F1F70197D9F7EFCFF894FFCFC1
:00000001FF
